:020000000150AD
:02000B00618F03
:03001B0041E83287
:0100230032AA
:100050007590FF75B0FF75816F75220175892575E3
:100060008D9CD28E758C00758A00752500C28CD34C
:10007000D2A9D2ABD2AFD2BB75301400C202C20338
:10008000C204C205C206C20775313275320A753321
:1000900000751800751900751A00E52FC394727069
:1000A00004A201400BD3752F72752E01D20180027C
:1000B000052EE52EB40118D28C75260C75272675F1
:1000C0002827752920752A01752B207F0A21F6B46F
:1000D000021CD28CD202D20475260F7527297528EE
:1000E0000E752920752A02752B207F0A21F6B4038C
:1000F0001CD28CD202C20575260F75272975280ED1
:10010000752920752A03752B207F0A21F6B404294E
:10011000751BFF751CFFD28CD20575262375270E23
:10012000752829752920752A04752B207F01851CC7
:100130008C851B8A75330021F6B40529751BF6756D
:100140001CFFD28CD20575262375270E75282975BC
:100150002920752A05752B207F01851C8C851B8A1B
:1001600075330021F6B40629751B9C751CFFD28CD3
:10017000D20575262375270E752829752920752A1D
:1001800006752B207F01851C8C851B8A7533002109
:10019000F6B40729751B17751CFCD28CD205752681
:1001A0002375270E752829752920752A07752B2098
:1001B0007F01851C8C851B8A75330021F6B40829C4
:1001C000751BEF751CD8D28CD20575262375270EAA
:1001D000752829752920752A08752B207F01851C13
:1001E0008C851B8A75330021F6C201C2AF7590FF62
:1001F00075B0FF4387027DFF7EFFDDFEDEFCDFFA88
:10020000410200300533300612152EE52EC206B429
:100210000305752E048019E52E210D300712052ED9
:10022000E52EC207B40905752E088004E52E210DC0
:10023000E533C394234002D206E52EB4010591476D
:100240000202E5B4021030030D71F271C0914D71DC
:10025000D1C2030202E5B4031330031071F271C07E
:10026000914D432A1071D1C2030202E5B404157501
:100270001BFF751CFF30030C914DC203432A107104
:10028000D10202E5B40515751BF6751CFF30030C91
:10029000914DC20343291071D10202E5B4061575D0
:1002A0001B9C751CFF30030C914DC2034328107139
:1002B000D10202E5B40715751B17751CFC30030C41
:1002C000914DC20343271071D10202E5B4081575A0
:1002D0001BEF751CD830030C914DC20343261071DF
:1002E000D10202E500004102C0E0C0D0C0003005EC
:1002F00014C2AF0518E518700C0519E5197006D27F
:1003000006051AE51AD2AFD5304E753014D5312A0C
:100310007531320533200409D5321F75320A300297
:1003200019C28CC28EA98AAA8CAB25758A00D28C80
:10033000D28E758C00752500D203D5220375220656
:1003400090035FE5222425F8E69375B0FFF59090C1
:100350000389E5221493F5B0D000D0D0D0E03288E4
:10036000BB1C192B49489B08090A68CC384C4E80A5
:10037000B314112341409300010260C4304446FF8E
:100380007F0F0E787CFB6CF77E7FDFF7FEFDFB2096
:100390000503052532851B8A851C8CA918AA19AB73
:1003A0001AC0E0C0D0EA54F84B7002D207D0D0D0C7
:1003B000E0751800751900751A00753300D2033204
:1003C00079007A007B007C0078347E0A9109DEFC9B
:1003D000227400B5261B752620B52715752720B574
:1003E000280F752820B52909752920B52A03752AF3
:1003F0002022C0017951784E7E1BE6F71819DEFAEB
:10040000D0E0F5348A358B3622E629F908E63AFA47
:1004100008E63BFBE43CFC0822858A23858C24E526
:1004200023540FF52BE523C4540FF52AE524540F6C
:10043000F529E524C4540FF528E525540FF527E5E3
:1004400025C4540FF52622A98AAA8CAB257806006C
:10045000EB54F0C475F00A84C4FCE5F0C4F5F0EB8D
:10046000540F25F075F00A844CFBE5F0C4F5F0EA72
:1004700054F0C425F075F00A84C4FCE5F0C4F5F02E
:10048000EA540F25F075F00A844CFAE5F0C4F5F053
:10049000E954F0C425F075F00A84C4FCE5F0C4F515
:1004A000F0E9540F25F075F00A844CF9AC0074267D
:0B04B0002814F8E5F0F6A804D8952207
